:030000000219FDE5
:03000B000200A848
:03002B0002015A75
:03005B000202EBB3
:030073000202D8AE
:1000800002030406080C10182030406080040608A3
:100090000C10182030406080A0C00003070F1F051F
:1000A000050D050305030302C2AFC0D0C0E0206206
:1000B00014E5256009E473E525F4F58AD262D0E001
:1000C000D0D0D2AF3285268AC262E526F4602F30C6
:1000D000682520720DD0E0D0D0C293C295C297D2CD
:1000E000AF32C293C295C297206F0C206509740A83
:1000F000D5E0FDE57B4290D0E0D0D0D2AF32758A1A
:1001000000C28DD26201F701B7306805206502D2C6
:100110009301B7306805206502D29501B7306805B4
:10012000206502D29701B7C29230680A2065077431
:1001300008D5E0FDD29301B7C29430680A20650764
:100140007408D5E0FDD29501B7C29630680A2065E3
:10015000077408D5E0FDD29701B7C2AFC2AD53E630
:10016000EFC0D0C0E0D2D3D2AFC2CEE52A60072024
:10017000744F152A21C17800790020742EE5803053
:100180007E01F430E30278FF53DACF207E0343DAB6
:1001900020307E0343DA10C2D8C271E580307E0180
:1001A000F430E30279FFC3E89970CB306103752A1C
:1001B00018207403752A18885CD270E86003755F94
:1001C0000020740DE52B6004152B21D143DA01C208
:1001D000D82070024144A85C206102C270207431B2
:1001E000C3E894F0400374F0F8E8C4540F28F87999
:1001F00084B703024111C313C3138721200802C32C
:1002000013200A06C3C898F8411128F8500374FF58
:10021000F8C3E895655003E565F88822E52D540696
:100220006022206B1FE536C333C333F8E564C31384
:10023000C313F9C3952240028922E82522F52250F2
:10024000037522FF852224A824C3E524956140027A
:10025000A8618825E56670024188C3E8AA669A50BD
:1002600003E8FAE4F9EAC333FBE568F45B29400DDF
:100270002567F8E56760021567400B41880AC3E50A
:10028000679A5002056778FF8826C26FC3E52694F7
:10029000F84002D26F20CF0AD0E0D0D043E610D28F
:1002A000AD32C2CF053A7801E52A600530740215F7
:1002B0002AC3E55C94014005755F0041CE7560007E
:1002C000756900E55F2401F55F5003755FFFD0E0BD
:1002D000D0D043E610D2AD32C2AF53E67F7592FA6A
:1002E0007593FFC260759104D2AF32C2AF53E6EF8F
:1002F000C2ADC0D0C0E0C0F0D2D3D2AFA8FBA9FC41
:10030000C2D8307102615253DACF207E0343DA1033
:10031000307E0343DA20D271E580307E01F420E3A1
:1003200002612988278928A17F53DACF207E0343E1
:10033000DA20307E0343DA10C2D8C271307402A1D1
:100340006B7800E580307E01F430E302A16B885CBD
:10035000A15353DACF207E0343DA20307E0343DA01
:1003600010C271206102812B53DACF207E0343DA61
:1003700010307E0343DA20C2D8D27188578958C31F
:10038000E89555F8E99556F97B007E087A00C3E8B0
:10039000948CE994005005755B00811D882178A23A
:1003A000E6A8216055C3E894C8E994005008E4D257
:1003B000E4FB7A0A61F8C3E89468E994015008E420
:1003C000D2E3FB7A0F61F8C3E894D0E994025008B5
:1003D000E4D2E2FB7A1E61F8C3E894A0E9940550E8
:1003E00008E4D2E1FB7A3C61F8C3E89498E9940808
:1003F0005008E4D2E0FB7A787E00C3E89559FCE926
:10040000955AFD30E70AECF42401FCEDF43400FDCC
:10041000755B00C3EC9AED9E5003755B01885989AA
:100420005A8557558558567802A153C3E89527F841
:10043000E99528F9307C02A137307B02A137307A68
:1004400002A130207502814EE9FDE8FC816DE9C30F
:1004500013F9E813F8307902A130E9C313F9E8136E
:10046000F8307802A130E9C313FDE813FC20612CB9
:0F047000C3EC941CED940240028184ED701EC316
:10047F00EC94C850180529E52970021529C3E52900
:10048F00940A5002A16B755C00D270A16BE52960D4
:10049F000215297888E6F97400207F087896B90349
:1004AF0002789EE624FAFEE43400FFC3EC9EFCEDD6
:1004BF009FFD9208B90310A2085007207609D27643
:1004CF0081D6307602C276A2085016B9030DECF42D
:1004DF002401FCEDF43400FD0204F078007900A152
:1004EF0037B90315EC33FCED33FDC3EC940AFCED87
:1004FF009400FD50047C007D00C3EC94FFED94004C
:10050F00400678FF7900A137EC8572F0A4C5F0A200
:10051F00F733F87900400302055378FF790002059D
:10052F0053E9C313F9E813F8307C0EE9600278FF42
:10053F00C3E81338F8E43400F9C3E894FFE99400F2
:10054F00400278FF885CD270206102A16B741FF4A7
:10055F00552F4BF52FC274EB7002D274752A1830D9
:10056F007403752A0A306102A17F20740353DAFEE7
:10057F00207403752B06D0F0D0E0D0D0D2AD43E677
:10058F00103279010205AF79030205AF790A02052E
:10059F00AF791E0205AF79640205AF79C80205AFC6
:1005AF007817E4D5E0FDD8FAD9F6227A147B7802D1
:1005BF0005D67A107B8C0205D67A0D7BB40205D650
:1005CF007A0B7BC80205D6E573D5E001227902E4E8
:1005DF00C294D5E0FDD295D5E0FDC295D5E0FDD210
:1005EF0094D5E0FDE920E002D29330E002D297E506
:1005FF0073D5E0FDE920E002C29330E002C29774A8
:10060F0096D5E0FDD9C9EAF8D5E0FDD8FBDBB8C235
:10061F009422C37C007D0075F00005F0EA33FAEBFD
:10062F0033FB50F6EB13FBEA13FAC3E9FFE8FEE8DE
:10063F009AF8E99BF95004EFF9EEF8B3EC33FCEDBF
:10064F0033FDD5F0DFEDF9ECF822E889F08A20D2FE
:10065F00D4F8A9F07B0030F70B7BFFF42401F8E905
:10066F00F43400F9E88520F0A4ADF0F8E98520F026
:10067F00A4AFF0FEED2EF974003FFA7C04C3EA1329
:10068F00FAE913F9E813F8DCF48BF030F70AE8F421
:10069F002401F8E9F43400F9E889F0C2D4F8A9F09C
:1006AF002222C3E54113F9E54013F8C3E54498F856
:1006BF00E54599F9500CC3E89480E994FF40160280
:1006CF0006E8C3E8947FE9940050030206E8787FB8
:1006DF0079000206E8788079FF8849894A22E5493E
:1006EF002546F8E54A3547F9854A20E4300701F4F5
:1006FF003548FA30E709C3EA94F04015020726C3DC
:10070F00EA940F500302072678FF79FF7A0F02074A
:10071F0026780079007AF0C3E5249561500AC374F6
:10072F00019524500B020744E54A20E70E020744C7
:10073F00E54A30E706884689478A482278A5E6FACF
:10074F00C3E54933F8E54A33F9D159E930E70BC32B
:10075F00E89480E994FF4013E17EC3E8947FE99425
:10076F00005002E17E787F7900E17E788079FFE8A2
:10077F0020E715C3E52398F84009C3E89401400327
:10078F000207A578010207A5E8F424012523F84004
:10079F00030207A578FF884B2278A6E6FAA847A997
:1007AF0048D159E930E70CC3E89401E994FF4016AA
:1007BF000207D9C3E894FFE9940050030207D978E0
:1007CF00FF79000207D9780179FFE920E715C3E522
:1007DF004B98F84009C3E8940140030208007801E0
:1007EF00020800E8F42401254BF8400302080078C2
:1007FF00FF88242278FF20692879A1E76023E5414B
:10080F00601F74FF8541F0848539F0306A0375F0FD
:10081F0005A4F8C5F0600278FFC3E895645002A8FC
:10082F0064886322C3E5409440E5419401E5635039
:10083F0003140144046002F5632202084C2275E898
:10084F0090227883E6FF30EDF9A8BDA9BE0570C3ED
:10085F00E57094084052757000E9FA79A0E760449A
:0E086F00EA7007E571601B020885C3E8957109
:10087D006010E5715006600C140208910460F902D5
:10088D000891E571F571C394A8401B7561C0C394BF
:10089D00054013756180C39405400B756140C39489
:1008AD0005400375610075BB0122E561F460020529
:1008BD0061E570B4070375BB1E22743279A787F00A
:1008CD00A4C5F0A2F733F8C3E895614002A861888A
:1008DD00228824882588268864227540007541F079
:1008ED0022C2AF75C820A8CCA9CDAA3A30CF010A33
:1008FD0075C824D2AFAB3BAC3C883B893CC3E89B6D
:10090D00F8E99C206908F930660221FF2159AD3DB7
:10091D008A3DF9EA9DFA600678FF79FF213EAE3EE9
:10092D00AF3F8B3E8C3FA83BA93CC3E89EF8E99FA7
:10093D00F9C3E54113FBE54013FAE82AF540E93B1D
:10094D00F54150067540FF7541FF21A6AA40AB4108
:10095D00AC40AD417E047F02C3EB9404400D1E1FDD
:10096D00C3EB94084005206A021E1FC3ED13FDEC76
:10097D0013FCDEF7C3EA9CFAEB9DFBEF6009C3E9BC
:10098D0013F9E813F8DFF7EA28FAEB39FB8A408B05
:10099D004150067BFF8B408B41C3EB94025002D23A
:1009AD00663069047F0321D17892E6FFC3E5379461
:1009BD008240110FC3E53794A040010FC3EF940699
:1009CD0040027F057E02E541C4540FF9E541C45450
:1009DD00F0F8E540C4540F28F8C3E89EFAE99400F6
:1009ED00FB4009C3EA9402EB940050047A02E4FB45
:1009FD00414BAA40AB41EBC4FEEAC4540F4EFCC3BD
:100A0D00EA9CFAEB9400FBC3E813C313F8EA28FA47
:100A1D00EB3400FB8A408B41C3EB94024002C2666B
:100A2D007802EBC4FE7B00EAC4540F4EFAC3EA9879
:100A3D00FA4005C3940250027A027892E6FF3060C4
:100A4D0002414B855192855293D26043E680C3E4B7
:100A5D009AF8E49BF930660241D7E8FAE9FBD3E94D
:100A6D0013FDE813FC88518952C3EF94036038EFEE
:100A7D0020E00DE82CF8E93DF9ECFAEDFB020AA0B7
:100A8D00E828F8E939F9C3E82402F8E93400F97ADD
:100A9D00FE7BFFC3EF9403400E8A538B54884D8920
:100AAD004E8C4F8D50610B885389548A4D8B4E8CD3
:100ABD004F8D503069127553F07554FF754FF075A9
:100ACD0050FF7551F07552FF610BE8FAD3E813FC36
:100ADD008851C3EF94036020EF20E007E82CF8EC79
:100AED00FA41F7E8282402F87AFEC3EF9403400890
:100AFD008A53884D8C4F610B88538A4D8C4FE56816
:100B0D00C3335002646BF5683060026115753402B1
:100B1D00D26043E680E52D54066034A840A941C358
:100B2D00E913F9E813F8C3E913F9E813F830690488
:100B3D00E92440F9C2AF53E67F759100C3E498F5FF
:100B4D0094E499F595759104D26043E680D2AF2275
:100B5D00D264754300752000306C03752040020B84
:100B6D007CD264754300752040306C03752000788D
:100B7D00017901206620E52D54066002C2647914C6
:100B8D00E541C313700104F8C39414400278143086
:100B9D006904781B791B206010E543600C306903F4
:100BAD00D53404D26D812F711D0543E59E7005E589
:100BBD009B020BC3E59A5440B52002811930690997
:100BCD0008C3E89940011861A320640A08C3E89995
:100BDD004002617C61A3C264C2AF53E67F75910090
:100BED003066127594007595F8759104D26043E6E0
:100BFD0080D2AF617CE5417EFFC3334005C33340F6
:100C0D0001FEC3E49E759400F59561F6C3E533943A
:100C1D00015002617C306402617CD802812D61A398
:100C2D00C26DC2AF53E67F7591008553948554957F
:100C3D00759104854D92854E93D26043E680D2AF77
:100C4D00E52D54066008206A020533020C6B306DE9
:100C5D000D206C0A2064071581158102156122781B
:0F0C6D00003064027801E53775F007A4F9E5F06F
:100C7C0028F5F0E9A2F013A2F113A2F213F537C391
:100C8C0094785003753778C3E53795384008D265AA
:100C9C00C293C295C29730600281A2854F92855053
:100CAC0093D26043E68022207D19C2AF754202C206
:100CBC0094D292306202D297D2AF759F33759E0058
:100CCC00020EB5C2AF754202C294D296306202D205
:100CDC0093D2AF759F33759E00020EB530724320D0
:100CEC007D20C2AF754203900138757B10C297C24C
:100CFC0096306204D295A106D294D2AF759E23028F
:100D0C000EB5C2AF754203900138757B10C293C209
:100D1C0092306204D295A126D294D2AF759E220253
:100D2C000EB5207D17C2AF754203900113C29730E8
:100D3C006202D295D2AF759E23020EB5C2AF754238
:100D4C0003900113C293306202D295D2AF759E22EA
:100D5C00020EB5207D16C2AF754204C292D29630F7
:100D6C006202D295D2AF759E22020EB5C2AF754209
:100D7C0004C296D292306202D295D2AF759E2302F3
:100D8C000EB5307249207D23C2AF75420590012704
:100D9C00757B04C295C294306204D293A1ACD292FA
:100DAC00D2AF759F33759E00020EB5C2AF7542056A
:100DBC00900149757B40C295C294306204D297A1D0
:100DCC00CFD296D2AF759F33759E00020EB5207DA3
:100DDC001AC2AF754205900109C295306202D293D6
:100DEC00D2AF759F33759E00020EB5C2AF7542052A
:100DFC0090011DC2953062E8D297D2AF759F3375C2
:100E0C009E00020EB5207D16C2AF754206C296D268
:100E1C0094306202D293D2AF759E23020EB5C2AF4C
:100E2C00754206C292D294306202D297D2AF759EAE
:100E3C0022020EB5307244207D20C2AF7542019063
:100E4C000149757B40C293C292306204D297C15E55
:100E5C00D296D2AF759E22020EB5C2AF75420190EA
:100E6C000127757B04C297C296306205D293020E9D
:100E7C007FD292D2AF759E23020EB5207D17C2AFE2
:100E8C0075420190011DC293306202D297D2AF75A8
:100E9C009E22020EB5C2AF754201900109C2973075
:100EAC006202D293D2AF759E23C265229001077560
:100EBC007B00C293C295C297C292C294C296C26280
:100ECC0022788076FF0876FF0876FF0876FF087692
:100EDC00030876040876070876030876010876017D
:100EEC00788C76010876FF0876FF0876FF0876FF87
:100EFC000876FF0876030876FF0876FF0876FF0869
:100F0C0076250876D00876FA0876FA0876040876FC
:100F1C00FF08760108760008767A0876FF087601D5
:100F2C00087601087600087603087600227887E6B2
:100F3C00FFC272BF0302D2727888E6C394036008C2
:100F4C00C27DE630E102D27DC27E7889E630E102D4
:100F5C00D27EC3EF94026008758E01D273020F71BA
:100F6C00758E00C273227880E6149000809378A569
:100F7C00F67881E6149000809378A6F67886E614CD
:100F8C0090008D9378A7F67886E6F539C3940250D5
:100F9C0003753902789CE67538FFB402037538A0E6
:100FAC00B4030375388278A3E61490009A93F5661F
:100FBC00D1B822227896E6FA7897E6FB7888E6B4E0
:100FCC000305C3EB940EFB307F047A007BFFC3EB6D
:100FDC009AFCC3948250027C827572000572EC8577
:100FEC0072F0A4C3E5F0947D40F222D27FF1C012DE
:100FFC0005A01205A07A007B007C10120596E55C1A
:10100C002AFA74003BFBDCF37C04C3EB13FBEA13FE
:10101C00FADCF7FEC27F120FC022757C00757D00D2
:10102C00E5EF20E6037520000520903DFFE5201438
:10103C006006901FFF1460009304600375EF165355
:10104C00D9BF7581C043FF8012059175EF0643B27D
:10105C0003E5B3240220E70DF521E5B120E0068578
:0E106C0021B343B101120EB875800875A400BF
:10107A0075F1FF75D4F775900275A5FC75F2FC75CC
:10108A00D50075A0FD75A60275F30275D60075B078
:10109A00FF75A70175F4FF75E241120EB8E4F8F680
:1010AA00D8FD756801120ECD1215B278988673753F
:1010BA003001C2AF1205AA1205BA1205A01205C163
:1010CA001205A01205C81205A01216DB1205AA12F3
:1010DA0005AA1205A5C2AF757C00757D0078FA795C
:1010EA00FA308307D9FBD8F7021C00120F39120F06
:1010FA0072120FBF120FC078988673120EB87588D5
:10110A001075890275C82475910475D84075A8228E
:10111A0075B80275E690759B80759D00759A807505
:10112A009C0075D10E75BC5875BB0175BA1F75E860
:10113A0080120591D2AF12084975360053DACF20D2
:10114A007E0343DA20307E0343DA1043DA01C2D841
:10115A00C2711205AAD2617B037A0CE55B70077A29
:10116A000CDB030210DF1205A02070030210DFC29D
:10117A0070E55CC3940240E1E52F541F855E5DF57E
:10118A005EB55DD5DAD5C26153DACF207E0343DA84
:10119A0020307E0343DA10C2D8C27178A2E6700802
:1011AA00D274E52F54E0F52FC2757529001205A5F2
:1011BA00307409C3E529940A4002D275120596785B
:1011CA00023074027800C3E55C9840F0C2AF1205A1
:1011DA00BA1205BA1205BAD2AF1205AA754C00782E
:1011EA0088E6B4030241E5120596788CE6C39401B9
:1011FA0050030212E5E530C3940150030212E5756B
:10120A007CA5757DF1207435C3E55C94FF5003021B
:10121A0012E5C2AF1205CFD2AF1205A5C3E55C94A1
:10122A000150EFC2AF1205BA12059B1205BAD2AF2E
:10123A001205A5C3E55C94FF40E90217607F05D259
:10124A007F120FC01205A5C2AFC27F120FC0AE5CDB
:10125A00C3E55C947FD2AF500241F5120591C2AF4B
:10126A001205CFD2AFDFD8120FF7C3EE94057897E5
:10127A00F61205AA1216E37F0AD27F120FC01205D0
:10128A00A5C2AFC27F120FC0AE5CC3E55C947FD229
:10129A00AF50E4120591C2AF1205BA12059B1205AE
:1012AA00BAD2AFDFD4120FF7EE24037896F6F879A4
:1012BA0097E7C394824003985006E824827897F609
:1012CA001205AA1216001217121205A5120FC0C390
:1012DA00E55C94FF50024109021760757C00757D38
:1012EA0000C3E55C954C4003855C4C1205A578016A
:1012FA007988E7B403027805C3E55C98400221E9DE
:10130A00C2AF1205CF1205CF1205CFD2AF1205AA6E
:10131A00753000E4F531F5320531E531F4703F05F9
:10132A0032789AE67819146012783214600D787D52
:10133A0014600878FA146003753200C3E5329840E5
:10134A001D120EB8120591153275310078998673FF
:10135A00C2AF1205CFD2AF789886731205A51205CF
:10136A009BE52A700530740201DF78012074027847
:10137A0006C3E55C9840A17888E6C394036003122B
:10138A0005A5E52A70030210DFC2AF120EB8E4F514
:10139A0022F523F524F525F526F567D2AF7885E6FB
:1013AA00C333F565E4F544F545F546F547F548F5E3
:1013BA0070F52CF52DF53775700875BB1E12059161
:1013CA0012084D30EDFDA8BDA9BEE97001F888717B
:1013DA0012085175700875BB1E120F39C2AF7561BC
:1013EA00FF1208C7852261852262852263D2AF7502
:1013FA002201752401752501752601856069756AC2
:10140A00017888E6B40307C27D307602D27DD268BD
:10141A00D269753300120E11120E401208E7120833
:10142A00EE1208E71208EE1208E7120B6E1206B067
:10143A00120C6C120CB31208EE120B5D306E031212
:10144A0006B1206603120803306603120833120C31
:10145A006C120CE81208EE120B6E306E031206EDD7
:0F146A00120C6C120D5F1208EE120B5D306E0348
:1014790012074B120C6C120D8E1208EE120B6E3005
:101489006E031207A8120C6C120E111208EE120844
:101499004D120B5D120C6C120E401208511208EE1F
:1014A90030692F856461856462856069756A01792F
:1014B900187A0CC3E53399400CC269D26A8A35752A
:1014C90061FF0214DBC3E55C94014003021434029A
:1014D9001569306A25206C22E535147006C26AD276
:1014E9006B8134F535C3E55C94014003021434780B
:1014F90088E6C3940360030215697536007882791A
:10150900A4E760027803C3E55F985054307404E59A
:101519002A604D7888E6B40317207D05207607A157
:1015290039307602A139206C07D26C8564618173E8
:1015390078F0306C058564617820C3E541985002E4
:101549008134306C1BC26CC27D307602D27DD26A86
:1015590075351285646181340536E55C6002A16CDC
:10156900753600C2AF120EB87887E6FE7602120F02
:10157900397887EEF6E4F522F523F524F525F526E5
:10158900F565752C00752D00D2AF1205A5120EB8A0
:1015990078A4E66006D293D295D297307409C3E550
:1015A900369404400201DF611D901A0D782012164D
:1015B90042E520B45A0CA3121642E520B4A5030251
:1015C90015E0757CA5757DF1120ECD121600757C9E
:1015D90000757D000215FF901A0378807B0A1216A8
:1015E90042A308DBF9901A0F788C7B19121642A3D3
:1015F90008DBF9901A2822C2AF12168512166290DA
:101609001A00740E121647A37409121647A374150B
:10161900121647901A0378807B0A121646A308DB34
:10162900F9901A0F788C7B19121646A308DBF91268
:101639001698121676901A2822E493F622E6438F1A
:1016490001538FFDFFC3E583941C400122EF857C84
:10165900B7857DB7F0538FFE22438F02438F0185F3
:101669007CB7857DB7901A0DF0538FFC22901A0D27
:10167900745AD147901A0E74A5D147227A3079D07D
:101689007820901A40D142E520F709A3DAF7227AA7
:101699003079D0901A40E7D14709A3DAF922AB741F
:1016A900A875BB01027984BB02027985BB03027963
:1016B90086BB04027992BB05027987BB060279A32E
:1016C900BB0702799CBB08027988BB09027989E8C2
:1016D900F7227C051205AADCFB22C2AF1205BA1259
:1016E90005C11205C81205CF12059B1205BA1205CC
:1016F900C11205C81205CF12059B1205BA1205C100
:101709001205C81205CFD2AF22C2AF1205CF1205FA
:10171900C81205C11205BA12059B1205CF1205C8D8
:101729001205C11205BA12059B1205CF1205C8127E
:1017390005C11205BAD2AF22AE74AF75C2AF120598
:10174900BA1205BA1205BA12059BDEF21205CF12BA
:10175900059BDFF8D2AF22D1E3D1DBD1DB75740170
:10176900757501757600F1417C05AD5C1205AAC35A
:10177900ED955C70F5C3E55C9401400AC3E55C94A2
:10178900FF403202179CD1A7D100D1E3C2AF75EF58
:1017990016D1DBDCD50576C3E5769403500280C605
:1017A900D1DB0575E5741490009F93F808C3E575BE
:1017B90098500280AED1DBD1DB0574C3E574940A7D
:1017C9005002809C120ECDD100C2AF75EF16D1DB4D
:0319FD00021026AF
:101A00000E0915FFFFFFFF0304070301015AA5019B
:101A1000FFFFFFFFFF03FFFFFF25D0FAFA04FF01DE
:091A2000007AFF0101000300FF40
:101A400023506C6174696E756D31353041232020EF
:101A500023424C48454C4923463331302320202033
:101A60002020202020202020202020202020202076
:101C0000C2AFC2D353D9BF7581C043B20343FF8073
:101C1000752438752503B1DC7529A5752AF175E29F
:101C20004043F10853A4F775D4FFD2837DFA7803BB
:101C300079E67C10752200752300901DE97B0675FE
:101C400024987525013083028145208308D8FBD96B
:101C5000F9DCF781B7308308D8FBD9F9DCF781B715
:101C6000B19CE493A3C39A6004DDC381B7DBDBB10D
:101C70008E6002812E7B08E493FAA3B16FDBF87AC1
:101C800030B16F752200752300B18EEAFCEBFDC305
:101C9000ED94FE400EB18E8A278B28ED30E0048A49
:101CA000828B83B18E7AC270D8C3ED94FE601950D6
:101CB000CEBD002BEC600F7520007521FF7529004B
:101CC000752A000200008100A827A9280809D80465
:101CD000D90281DCB192EA89AAF281CE0D81A3C337
:101CE000ED94035053EDA2E092007AC5C3E58294CF
:101CF00000E583941C508A200010438F02438F011B
:101D00008529B7852AB7F0300029A827A92808090E
:101D1000438F01538FFDD804D902A133C3E58394C7
:101D20001C4003A3A11689AAE28529B7852AB7F02A
:101D3000A3A116538FFC817F7AC1BD030CE493A34A
:101D4000FAB153DCF8B14B817F8181AA22AB23B178
:101D50006FEBFAEA6222752608C3E52313F523E543
:101D60002213F52250066323A0632201D526EAB18F
:101D7000DCB1DC75260AEAF4200102D283300102CC
:101D8000C283B1DCC3134002C201D526EB22B1925B
:101D9000EAFB208302A192308302A197752608AE48
:101DA00024AF25C3EF13FFEE13FEB1E0B1DCC3EAAD
:101DB000133083024480FA30E703632201C3E52332
:101DC00013F523E52213F52250066323A0632201B5
:101DD000D526D9E52265236523F52222AE24AF2539
:101DE0000E0FDEFEDFFCD20122424C48656C6934E6
:071DF000373164F310060116
:00000001FF
